:020000040000FA
:04000000CC303A289E
:08000800A000030EA100831209
:1000100005191028831601178312B23081002B288E
:1000200083160113831203140B190310A80DA90DD5
:10003000AA0DAB0DAC0DAC16FF302C02031D2B2806
:10004000FA302B02031D2B2831152A08AF0029088E
:10005000AE002808AD008B100B11210E8300A00EFE
:04006000200E090065
:0C007400203084008001840A6030040207
:10008000031C3C281230B0009D2183160C308505DE
:1000900087018312850187010730990000309A009B
:1000A000103083168E008312603083168F00831207
:1000B0000030831691008312C830831681008312AA
:1000C00031309000003083168C00831210308B008A
:1000D000831600309B001C141A088312BC00831680
:1000E00010309B001C141A088312BD002E228101BF
:1000F0008E018F010B118B100B108C018B178E2032
:1001000031199120B30B8C28031085190314B90DF4
:10011000F03039020319162185227F28640032103D
:10012000080031110130B7008B13203037078316D8
:100130009B001C141A088312A40010303707831682
:100140009B001C141A088312A300A6000230A60606
:100150000030370783169B001C141A088312A20074
:10016000A7000130A7068B17321CBC2822090339CF
:10017000A200A309A409A50924082F02031D102920
:1001800023082E02031D102922082D02031D102909
:1001900001303702031DD1283D18D1283D143E14EB
:1001A000AA2102303702031DDA28BD18DA28BD144F
:1001B0003E14B62103303702031DE3283D19E3281E
:1001C0003D153E14C22104303702031DEC28BD1931
:1001D000EC28BD153E14CE2105303702031DF5284D
:1001E0003D1AF5283D163E14DA2106303702031D6C
:1001F000FE28BD1AFE28BD163E14E5210730370241
:10020000031D07293D1B07293D173E14F021083027
:100210003702031D1029BD1B1029BD173E14FB21F9
:10022000B70A093037020318080094280130B600D5
:10023000B300B400B500B70085018701B1138E206B
:10024000B30B4E29031085190314B90DF030390290
:1002500003197529B40B4E29013037020319062200
:100260000230370203190B22033037020319102220
:1002700004303702031915220530370203191A22F8
:100280000630370203191F220730370203192422D0
:1002900008303702031929229630B400311D1F2976
:1002A0003111321C58292D090339AD00AE09AF09AF
:1002B0002F1C1F298E018F010C1C1F290C102E1EB4
:1002C0001F298B1320303707BB002F08BA00882165
:1002D00010303707BB002E08BA00882100303707DE
:1002E000BB002D08BA0088218B1785018701B70A4A
:1002F000B60109303702031C1F292E2208003E1CBC
:1003000008003E101030BB003D08BA0088210800EC
:100310008B133A0883161C159A0083123B08831628
:100320009B0055309D00AA309D009C1464009C18D1
:1003300096291C1183128B170800FF30C800CA15BC
:10034000CB15CC15CD15CE15CF15D015D115D21591
:10035000D3150800F130BD05FF30DE051130C405AE
:10036000C0000030C200C6005F100800F230BD05BA
:10037000FF30DE050230C405C0000030C200C600F8
:100380005F100800F430BD05FF30DE050630C405FF
:10039000C0000030C200C6005F100800F830BD0584
:1003A000FF30DE051830C405C0000030C200C600B2
:1003B0005F1008001F30BD05C030DE058830C50560
:1003C000C1000030C300C70008002F30BD05C03099
:1003D000DE051030C505C1000030C300C7000800AD
:1003E0004F30BD05C030DE053030C505C1000030DE
:1003F000C300C70008008F30BD05C030DE05C03027
:10040000C505C1000030C300C700080010308506D4
:100410000230870608002030850600308706080075
:10042000213085060030870608000230850602303C
:1004300087060800003085060C308706080000306B
:1004400085060130870608000030850621308706C2
:100450000800003085061830870608003D18AA21DC
:10046000BD18B6213D19C221BD19CE213D1ADA2190
:10047000BD1AE5213D1BF021BD1BFB210800B60183
:10048000B301B4013C1C472ABC01BC14492ABC017D
:100490003C143C08B60064004D2A4E2A4F2A502ACC
:1004A000512AFF30B41B8500B41F8501B30B4B2AC2
:1004B000B40B4B2A0310B60CB608031D4B2A0030B0
:1004C000BB003C08BA008821080005125C1805161C
:1004D000DC1C8512DC1885165C1D05105C190514E2
:1004E000DC1D8510DC1985145C1E87105C1A8714CE
:1004F000DC1E0711DC1A07155C1F07105C1B0714B4
:10050000DC1F8712DC1B871608008F080319080000
:100510008F0178308E00C80FAF2CC80A441CB52A52
:10052000461CA62ACA1C972ACA014A15C32A4A1D74
:100530009C2ACA01CA15C32ACA1DA12ACA014A1681
:10054000C32A4A1EC32ACA01CA14C32A4A1DAB2A97
:10055000CA014A16C32ACA1DB02ACA014A16C32AAA
:100560004A1EC32ACA01CA14C32ACA1CBA2ACA010B
:100570004A15C32A4A1DBF2ACA01CA15C32A4A1EE0
:10058000C32ACA014A15C41CEA2AC61CDB2ACB1C92
:10059000CC2ACB014B15F82A4B1DD12ACB01CB1508
:1005A000F82ACB1DD62ACB014B16F82A4B1EF82A67
:1005B000CB01CB14F82A4B1DE02ACB014B16F82AAD
:1005C000CB1DE52ACB014B16F82A4B1EF82ACB018E
:1005D000CB14F82ACB1CEF2ACB014B15F82A4B1D64
:1005E000F42ACB01CB15F82A4B1EF82ACB014B1568
:1005F000441D1F2B461D102BCC1C012BCC014C1570
:100600002D2B4C1D062BCC01CC152D2BCC1D0B2BD3
:10061000CC014C162D2B4C1E2D2BCC01CC142D2B8C
:100620004C1D152BCC014C162D2BCC1D1A2BCC019F
:100630004C162D2B4C1E2D2BCC01CC142D2BCC1C51
:10064000242BCC014C152D2B4C1D292BCC01CC156A
:100650002D2B4C1E2D2BCC014C15C41D552BC61D0E
:10066000462BCD1C372BCD014D155F13632B4D1D34
:100670003C2BCD01CD15632BCD1D412BCD014D164E
:10068000632B4D1E632BCD01CD14632B4D1D4B2BC6
:10069000CD014D16632BCD1D502BCD014D16632B77
:1006A0004D1E632BCD01CD14632BCD1C5A2BCD01D8
:1006B0004D15632B4D1D5F2BCD01CD15632B4D1EAD
:1006C000632BCD014D155F1B8C2B441E8C2B461EBE
:1006D0007D2BCE1C6E2BCE014E159A2B4E1D732BEF
:1006E000CE01CE159A2BCE1D782BCE014E169A2B0D
:1006F0004E1E9A2BCE01CE149A2B4E1D822BCE016C
:100700004E169A2BCE1D872BCE014E169A2B4E1EBF
:100710009A2BCE01CE149A2BCE1C912BCE014E15C6
:100720009A2B4E1D962BCE01CE159A2B4E1E9A2B30
:10073000CE014E15C51DC12BC71DB22BCF1CA32B3F
:10074000CF014F15CF2B4F1DA82BCF01CF15CF2B8E
:10075000CF1DAD2BCF014F16CF2B4F1ECF2BCF016F
:10076000CF14CF2B4F1DB72BCF014F16CF2BCF1D43
:10077000BC2BCF014F16CF2B4F1ECF2BCF01CF1449
:10078000CF2BCF1CC62BCF014F15CF2B4F1DCB2B03
:10079000CF01CF15CF2B4F1ECF2BCF014F15451EAD
:1007A000F62B471EE72BD01CD82BD0015015042C5C
:1007B000501DDD2BD001D015042CD01DE22BD00113
:1007C0005016042C501E042CD001D014042C501DA3
:1007D000EC2BD0015016042CD01DF12BD00150165B
:1007E000042C501E042CD001D014042CD01CFB2B44
:1007F000D0015015042C501D002CD001D015042C14
:10080000501E042CD0015015C51E2B2CC71E1C2CAD
:10081000D11C0D2CD1015115392C511D122CD10197
:10082000D115392CD11D172CD1015116392C511E3F
:10083000392CD101D114392C511D212CD101511643
:10084000392CD11D262CD1015116392C511E392C91
:10085000D101D114392CD11C302CD1015115392C96
:10086000511D352CD101D115392C511E392CD101F6
:100870005115451F612C471F522CD21C432CD2010D
:100880005215DF136F2C521D482CD201D2156F2C3C
:10089000D21D4D2CD20152166F2C521E6F2CD2013C
:1008A000D2146F2C521D572CD20152166F2CD21D10
:1008B0005C2CD20152166F2C521E6F2CD201D21416
:1008C0006F2CD21C662CD20152156F2C521D6B2C32
:1008D000D201D2156F2C521E6F2CD2015215DF1B84
:1008E000982CC51F982CC71F892CD31C7A2CD30198
:1008F0005315A62C531D7F2CD301D315A62CD31D25
:10090000842CD3015316A62C531EA62CD301D3142A
:10091000A62C531D8E2CD3015316A62CD31D932C1D
:10092000D3015316A62C531EA62CD301D314A62CE8
:10093000D31C9D2CD3015315A62C531DA22CD301DF
:10094000D315A62C531EA62CD30153157F21400886
:10095000C4004108C5005F18DF145F1CDF104808A1
:10096000C9000C304A05031D05120C304B05031D50
:1009700085120C304C05031D05100C304D05031D70
:1009800085100C304E05031D87100C304F05031DDC
:1009900007110C305005031D07100C305105031DC5
:1009A00087120C305205031D07120C305305031D2E
:1009B000871149080E020318092D12304A05031D3C
:1009C000051612304B05031D851612304C05031D0C
:1009D000051412304D05031D851412304E05031DFC
:1009E000871412304F05031D071512305005031DE3
:1009F000071412305105031D871612305205031DCE
:100A0000071612305305031D8715FF3048020319DE
:100A100008008F08031D08008E2049080E02031CE1
:100A2000092D18304A05031D051206304A05031D1D
:100A3000051618304B05031D851206304B05031DA6
:100A4000851618304C05031D051006304C05031D96
:100A5000051418304D05031D851006304D05031D86
:100A6000851418304E05031D871006304E05031DF2
:100A7000871418304F05031D071106304F05031D5D
:100A8000071518305005031D071006305005031DCB
:100A9000071418305105031D871206305105031D38
:100AA000871618305205031D071206305205031D24
:100AB000071618305305031D871106305305031D13
:040AC000871508008E
:084000000400030002000600A9
:02400E00CC33B1
:10420000010078007A007C007E007B0079007F004E
:104210007D007A0078007E007C007D007F00FF003A
:104220000200F200F600FA00FE00F200F600FA00CA
:10423000FE00F200F600FA00FE00F200F600FF00B9
:10424000FF00050005000500050009000900090040
:1042500009000D000D000D000D0011001100FF0000
:104260000100FF00FF00FF00FF00FF00FF00FF0054
:10427000FF00FF00FF00FF00FF00FF00FF00FF0046
:10428000FF00FF00FF00FF00FF00FF00FF00FF0036
:10429000FF00FF00FF00FF00FF00FF00FF00FF0026
:1042A000FF00FF00FF00FF00FF00FF00FF00FF0016
:1042B000FF00FF00FF00FF00FF00FF00FF00FF0006
:1042C000FF00FF00FF00FF00FF00FF00FF00FF00F6
:1042D000FF00FF00FF00FF00FF00FF00FF00FF00E6
:1042E000FF00FF00FF00FF00FF00FF00FF00FF00D6
:1042F000FF00FF00FF00FF00FF00FF00FF00DD00E8
:00000001FF
